:100000000C9437010C9454010C9454010C94540139
:100010000C9454010C9454010C9454010C9454010C
:100020000C9454010C9454010C9454010C945401FC
:100030000C94CF120C9454010C9454010C94540160
:100040000C9454010C94B3050C9480190C94E41195
:100050000C946E120C9454010C9454010C945401A1
:100060000C9454010C9454010C9454010C945401BC
:100070004570692D4F5344205665722E302E392E0F
:10008000322E310000416B7475656C6C65732053C2
:10009000657474696E67000053657474696E6720D7
:1000A000200000486F6568656E73656E736F72201F
:1000B00000004853206D697420536368616C746557
:1000C0007220000048656164696E6720486F6C6447
:1000D0002000004B6F6D706173732000004B6F6DDB
:1000E0007061737320666978200000475053204187
:1000F0006B74697620000041636873656E6B6F7086
:1001000070656C756E67200000447265687261747A
:100110006520626567722E2000004665686C657216
:100120002046433C2D3E4F5344200000556E7465DD
:10013000727370616E6E756E672000004B65696E3C
:10014000652053657474696E672D416E7A656967C1
:1001500065000050432F425420616B7469760000A3
:1001600055656265726E65686D65204C65747A745C
:1001700065732053657474696E6700004B65696E22
:1001800065204465766976652D416E7A6569676597
:10019000000050432F425420616B74697600005573
:1001A000656265726E65686D65204C65747A74650C
:1001B000732044657669636500004F4E00002D2D65
:1001C0002D000044657669636520756E6420566570
:1001D0007273696F6E736162667261676500004475
:1001E000656369766520202020203D200000465769
:1001F0002D56657273696F6E203D200000464300E6
:10020000004E43000046432D6F6C642046570000AB
:100210004550492D4D656E750050616C0050432F5F
:100220004254004B656E6E756E670052432D4265F9
:100230007472696562004550492D5374726F6D0088
:1002400045786974004F4E002D2D0076767D7676C8
:100250007A76767E76767776767B76767876767C24
:1002600076767976767D76767A76767E7600112445
:100270001FBECFEFD4E0DEBFCDBF11E0A0E0B1E004
:10028000E4E1F5E302C005900D92A039B107D9F77A
:1002900013E0A0E9B1E001C01D92AB3AB107E1F76C
:1002A0000E9464010C94881A0C94000086E981BBBA
:1002B0008FE084BBAC9AAD9A8EE28ABB80EB87BBA1
:1002C000C69AD99ADD9A08951092D8011092D40155
:1002D0001092D901E199FECF80E090E09FBB8EBBE8
:1002E000E09A8DB380939701E199FECF81E090E091
:1002F0009FBB8EBBE09A8DB380930001E199FECF46
:1003000082E090E09FBB8EBBE09A8DB38093980112
:10031000E199FECF87E190E09FBB8EBBE09A8DB361
:100320008093A501E199FECF88E190E09FBB8EBB51
:10033000E09A8DB38093BE01E199FECF8AE190E00F
:100340009FBB8EBBE09A8DB380930901E199FECFEC
:1003500089E190E09FBB8EBBE09A8DB38093BA0198
:10036000E199FECF8BE190E09FBB8EBBE09A8DB30D
:100370008093990120910001213079F49EE09093BF
:10038000030187E08093040186E8809305012093B0
:100390000601909307018CE00EC09CE0909303014E
:1003A00085E0809304018AE48093050110920601A0
:1003B000909307018AE0809308010E94A8170E9489
:1003C00056010E94AC0580919701813019F40E947A
:1003D000BF1002C00E94AF107894A89A0E94E20455
:1003E0000E9414060E94070A80919901882311F047
:1003F0000E94470A8091C301882311F00E949D1337
:100400000E94470A80919901813011F40E94D0190D
:100410000E9490118091B601813021F41092B601B2
:100420000E9440188091DD01813021F41092DD019D
:100430000E94DD0D809192018130E9F410929201C9
:100440008091D801882389F48091BA01843069F4BD
:1004500080919701882349F480919A01813029F491
:1004600080E363E64AE00E943E110E94C2120E94AD
:10047000C7120E94EB1480919901813031F4809170
:10048000DE01813011F40E94DB19809195018130E9
:10049000E1F48091D8018823C1F4AA9A0E94040F44
:1004A0000E9467090E947C088091C101882321F085
:1004B0000E943B130E94C50A8091C201882311F05B
:1004C0000E94F0170E949C0AAA98809190018130A6
:1004D00069F58091D801882349F5109290018091A7
:1004E000A501882321F080910201833014F00E943D
:1004F000760A8091A2019091A30101969093A301A5
:100500008093A2010197CB9769F48091A00190910B
:10051000A10101969093A1018093A0011092A301E3
:100520001092A2010E94550C0E949F0D8091910192
:10053000813009F06FCF8091D801882309F06ACF0C
:100540001092910180919901813039F48091DE01FE
:10055000882319F481E00E94DB190E94100A80911F
:10056000C301882309F456CF0E94F5130E9460143A
:1005700051CF782FD99827E030E041E050E0DB9868
:100580000000000000000000CA01022E02C0880F17
:10059000991F0A94E2F7872311F0DA9A01C0DA98DA
:1005A0000000000000000000DB9A000000000000D6
:1005B0000000215030408FEF2F3F380701F727E030
:1005C00030E041E050E0DB98000000000000000057
:1005D000CA01022E02C0880F991F0A94E2F78623EF
:1005E00011F0DA9A01C0DA98000000000000000063
:1005F000DB9A0000000000000000215030408FEF27
:100600002F3F380701F7DB98DA98D99A089584E0EC
:1006100064E00E94B90280E06CE40E94B90210928A
:100620009201809192018823E1F38CE66AE00E94B6
:10063000B90285E060E00E94B90208951F9380919D
:10064000BA01823051F40E94CF1010929001809133
:1006500090018823E1F31092900182E661E74FEF69
:100660000E943E111092900110E00DC08091950102
:10067000813011F40E94040F80919001813019F4AF
:100680001092900111E08091C001882311F4112390
:1006900069F38091BA01823011F40E94161111237E
:1006A00009F0D9C080919B038093090180918A034E
:1006B0008093BE012091BE01E199FECF88E190E0D8
:1006C0009FBB8EBB2DBB0FB6F894E29AE19A0FBE8A
:1006D00020910901E199FECF8AE190E09FBB8EBB9A
:1006E0002DBB0FB6F894E29AE19A0FBE82E061E06A
:1006F00045E850E00E943F0E82E062E048E950E0A9
:100700000E943F0E82E064E043EA50E00E943F0E08
:1007100082E065E042EB50E00E943F0E82E066E03E
:1007200044EC50E00E943F0E82E067E043ED50E071
:100730000E943F0E82E068E04DED50E00E943F0EC7
:1007400082E069E04BEE50E00E943F0E82E06AE0FA
:1007500047EF50E00E943F0E82E06BE04CE251E038
:100760000E943F0E4091BC015091BD0184E162E0C6
:100770000E94B20D8091BE0180FF05C084E164E05B
:100780004AEB51E004C084E164E04EEB51E00E948A
:100790003F0E8091BE0181FF05C084E165E04AEB18
:1007A00051E004C084E165E04EEB51E00E943F0E51
:1007B0008091BE0182FF05C084E166E04AEB51E012
:1007C00004C084E166E04EEB51E00E943F0E809150
:1007D000BE0183FF05C084E167E04AEB51E004C03D
:1007E00084E167E04EEB51E00E943F0E8091BE0134
:1007F00084FF05C084E168E04AEB51E004C084E175
:1008000068E04EEB51E00E943F0E8091BE0185FFF3
:1008100005C084E169E04AEB51E004C084E169E08D
:100820004EEB51E00E943F0E8091BE0186FF05C055
:1008300084E16AE04AEB51E004C084E16AE04EEBF7
:1008400051E00E943F0E4091090184E16BE050E0CD
:100850000E94B20D20C082E062E045E850E00E94B4
:100860003F0E82E065E04AE151E00E943F0EE199CF
:10087000FECF88E190E09FBB8EBBE09A8DB3809362
:100880008A03E199FECF8AE190E09FBB8EBBE09A9C
:100890008DB38093090190918A03892F8170809391
:1008A000C101892F88708093C201892F8072809343
:1008B000C30194709093C4011F9108951F93809178
:1008C00090018823E1F31092900183E666E740E00F
:1008D0000E943E1110E00DC080919501813011F40D
:1008E0000E94E70E80919001813019F410929001DE
:1008F00011E08091BB01882311F4112369F31123C6
:1009000009F054C082E062E043EC51E00E943F0EE7
:1009100082E064E04FED51E00E943F0E82E066E02D
:100920004EEE51E00E943F0E8091BA01813031F4C9
:100930008EE064E04DEF51E00E943F0E8091BA01DD
:10094000823031F48EE064E041E052E00E943F0EDC
:100950008091BA01843031F48EE064E045E052E0E9
:100960000E943F0E409144038EE066E050E00E94FA
:10097000B20D4091450380E166E050E00E94B20D67
:100980004091460383E166E050E00E94B20D209161
:10099000BA01E199FECF89E190E09FBB8EBB2DBBF0
:1009A0000FB6F894E29AE19A0FBE0AC0E199FECF21
:1009B00089E190E09FBB8EBBE09A8DB38093BA0132
:1009C0001F9108950E94070383E66FE644E60E94A4
:1009D0003E1110929001809190018823E1F387E00D
:1009E00062E040E750E00E943F0E0E941506109220
:1009F0009001809190018823E1F310929001809101
:100A000090018823E1F31092900180919001882356
:100A1000E1F31092900184E064E00E94B90280E06A
:100A20006CE40E94B90280919701882319F40E9416
:100A30005E041CC082E062E04CE751E00E943F0E81
:100A400082E064E042E951E00E943F0E82E066E00D
:100A50004FE951E00E943F0EE199FECF89E190E01D
:100A60009FBB8EBBE09A8DB38093BA0180919001B9
:100A70008823E1F310929001809190018823E1F3A3
:100A80001092900184E064E00E94B90280E06CE47E
:100A90000E94B90280919701882319F40E941E03D5
:100AA00026C082E062E04CE351E00E943F0E82E00B
:100AB00064E043E551E00E943F0E82E066E040E6DC
:100AC00051E00E943F0EE199FECF88E190E09FBB8C
:100AD0008EBBE09A8DB38093BE01E199FECF8AE18F
:100AE00090E09FBB8EBBE09A8DB38093090180910B
:100AF000BA01823029F483E66FE64AE00E943E1193
:100B00008091BA01813029F482E664E64AE00E94CD
:100B10003E11809190018823E1F310929001809121
:100B200090018823E1F31092900180919001882335
:100B3000E1F310929001809190018823E1F31092EB
:100B40009001809190018823E1F31092900184E05C
:100B500064E00E94B902089582E083BF82E48EBD02
:100B60008AE089BF08951F920F920FB60F92112449
:100B70008F939F93809194018F5F809394018091D4
:100B80009401883449F591E0909393011092940177
:100B90008091A1038F5F8093A1038091A10384368C
:100BA00031F41092A1039093900190939101809160
:100BB000A103823319F481E0809391018091A00315
:100BC0008F5F8093A0038091A0038A3029F4109254
:100BD000A00381E0809392019F918F910F900FBEAF
:100BE0000F901F901895982F80538A3010F020E0B6
:100BF00005C0903311F42AE001C0282F892F8154B9
:100C00008A3110F4292F2653892F81568A3110F406
:100C1000292F2C539D3211F429E403C09E3209F48C
:100C200021E4822F08950895089585E060E00E94F0
:100C3000B90286E063E80E94B90287E060E90E9499
:100C4000B90285E060E00E94B90286E064E80E9493
:100C5000B90287E061E90E94B90285E060E00E9484
:100C6000B90286E065E80E94B90287E062E90E9465
:100C7000B90285E060E00E94B90286E066E80E9461
:100C8000B90287E063E90E94B90285E060E00E9452
:100C9000B90286E067E80E94B90287E064E90E9431
:100CA000B90285E060E00E94B90286E068E80E942F
:100CB000B90287E065E90E94B90285E060E00E9420
:100CC000B90286E069E80E94B90287E066E90E94FD
:100CD000B90285E060E00E94B90286E06AE80E94FD
:100CE000B90287E067E90E94B90285E060E00E94EE
:100CF000B90286E061EA0E94B90287E068E90E94D1
:100D0000B90285E060E00E94B90286E062EA0E94D2
:100D1000B90287E069E90E94B90285E060E00E94BB
:100D2000B90286E063EA0E94B90287E06AE90E949C
:100D3000B90285E060E00E94B90286E064EA0E94A0
:100D4000B90287E06BE90E94B90285E060E00E9489
:100D5000B90286E065EA0E94B90287E06CE90E9468
:100D6000B90285E060E00E94B90286E066EA0E946E
:100D7000B90287E06DE90E94B90285E060E00E9457
:100D8000B90286E067EA0E94B90287E06EE90E9434
:100D9000B90285E060E00E94B90286E068EA0E943C
:100DA000B90287E06FE90E94B90285E060E00E9425
:100DB000B90286E06FEB0E94B90287E060EA0E9408
:100DC000B90285E060E00E94B90286E060EC0E9412
:100DD000B90287E061EA0E94B90285E060E00E9402
:100DE000B90286E061EC0E94B90287E062EA0E94E3
:100DF000B90285E060E00E94B90286E062EC0E94E0
:100E0000B90287E063EA0E94B90285E060E00E94CF
:100E1000B90286E063EC0E94B90287E064EA0E94AE
:100E2000B90285E060E00E94B90286E064EC0E94AD
:100E3000B90287E065EA0E94B90285E060E00E949D
:100E4000B90286E065EC0E94B90287E066EA0E947A
:100E5000B90285E060E00E94B90286E066EC0E947B
:100E6000B90287E067EA0E94B90285E060E00E946B
:100E7000B90286E06DED0E94B90287E068EA0E943F
:100E8000B90285E060E00E94B90286E06EED0E9442
:100E9000B90287E069EA0E94B90285E060E00E9439
:100EA000B90286E06FED0E94B90287E06AEA0E940B
:100EB000B90285E060E00E94B90286E060EE0E941F
:100EC000B90287E06BEA0E94B90285E060E00E9407
:100ED000B90286E061EE0E94B90287E06CEA0E94E6
:100EE000B90285E060E00E94B90286E062EE0E94ED
:100EF000B90287E06DEA0E94B90285E060E00E94D5
:100F0000B90286E063EE0E94B90287E06EEA0E94B1
:100F1000B90285E060E00E94B90286E064EE0E94BA
:100F2000B90287E06FEA0E94B90285E060E00E94A2
:100F3000B90286E06BEF0E94B90287E060EB0E9485
:100F4000B90285E060E00E94B90286E06CEF0E9481
:100F5000B90287E061EB0E94B90285E060E00E947F
:100F6000B90286E06DEF0E94B90287E062EB0E9451
:100F7000B90285E060E00E94B90286E06EEF0E944F
:100F8000B90287E063EB0E94B90285E060E00E944D
:100F9000B90286E06FEF0E94B90287E064EB0E941D
:100FA000B90285E061E00E94B90286E060E00E943B
:100FB000B90287E065EB0E94B90285E061E00E941A
:100FC000B90286E061E00E94B90287E066EB0E9408
:100FD000B9020895BF92CF92DF92EF92FF920F93E2
:100FE0001F93CF93DF937C01B62E8C0145E0C42E76
:100FF000D12CC80ED91E862F90E0EC01CC0FDD1F3E
:10100000C80FD91FCA5EDE4F0EC085E0612F0E9457
:10101000B90286E0602F0E94B90287E068810E94D1
:10102000B9020F5F1F4F0C151D0578F38701065F8E
:101030001F4F8FE090E0E80EF91E8B2D90E0EC0141
:10104000CC0FDD1FC80FD91FCA5EDE4F0EC085E072
:10105000612F0E94B90286E0602F0E94B90287E0EA
:1010600068810E94B9020F5F1F4F0E151F0578F3AC
:10107000DF91CF911F910F91FF90EF90DF90CF9074
:10108000BF900895EF92FF920F931F93CF93DF933A
:101090008C01EC0155E0E52EF12CE80EF91E0DC097
:1010A00085E06D2F0E94B90286E06C2F0E94B90284
:1010B00087E060E00E94B9022196CE15DF0580F33B
:1010C000E8012A96015F1F4F0DC085E06D2F0E9439
:1010D000B90286E06C2F0E94B90287E060E00E94AE
:1010E000B9022196C017D10780F3DF91CF911F91EC
:1010F0000F91FF90EF9008951F93CF93DF93C091CE
:101100004402D0914502D7FD12C0CE016AE070E0E2
:101110000E94751A182F16952091040130E0CE0117
:101120006AE070E00E94751A261B310918C0EE278C
:10113000FF27EC1BFD0BCF016AE070E00E94751ADF
:10114000182F16951C5F2091040130E02F5F3F4F50
:10115000CF016AE070E00E94751A260F311DE90187
:1011600075E0CC0FDD1F7A95E1F7220F331FC21B0C
:10117000D30B27968091120190911301C817D907BC
:1011800039F080911201909113010E94420804C02D
:101190008091C701811721F0CE01612F0E94EA07DB
:1011A0001093C701D0931301C0931201DF91CF9127
:1011B0001F910895CF92DF92EF92FF920F931F93AA
:1011C000CF93DF938C01E62E85E0612F0E94B90258
:1011D00086E0602F0E94B902CE2CDD2484E391E0EA
:1011E000C80ED91E87E0F60160810E94B902EEE1C7
:1011F000EE2EF12CE00EF11E85E06F2D0E94B9025B
:1012000086E06E2D0E94B90287E0F60160810E949F
:10121000B902E801CC54DF4F025F1E4F85E06D2F0D
:101220000E94B90286E06C2F0E94B90287E0F601A5
:1012300060810E94B9026E96C017D10779F7DF91DD
:10124000CF911F910F91FF90EF90DF90CF90089575
:10125000EF92FF920F931F93CF93DF937C0185E072
:101260006F2D0E94B90286E06E2D0E94B90287E0C0
:1012700060E00E94B9028701025E1F4F85E0612F86
:101280000E94B90286E0602F0E94B90287E060E008
:101290000E94B902E701CC54DF4F8701025F1E4F65
:1012A00085E06D2F0E94B90286E06C2F0E94B90282
:1012B00087E060E00E94B9026E96C017D10781F7FF
:1012C000DF91CF911F910F91FF90EF9008951F93A1
:1012D000CF93DF93E0914202F0914302F7FD14C0F7
:1012E000CF016AE070E00E94751A182F16951C5FF6
:1012F00080910501C82FD0E0CF016AE070E00E9424
:10130000751AC61BD10917C0222733272E1B3F0B86
:10131000C9016AE070E00E94751A182F1695809135
:101320000501C82FD0E02196C9016AE070E00E9453
:10133000751AC60FD11D8091140190911501C8171F
:10134000D90739F080911401909115010E94280964
:1013500004C08091C801811721F0CE01612F0E9445
:10136000DA081093C801D0931501C0931401DF91DE
:10137000CF911F91089585E060E00E94B90286E058
:101380006FEC0E94B90287E06CE80E94B90285E028
:1013900061E00E94B90286E06BE00E94B90287E03A
:1013A0006DE80E94B9020895EF92FF920F931F9388
:1013B000CF93DF937A019EE1699FB0011124680FFA
:1013C000711D8B01020F111D1092A203EB0115C0BC
:1013D00085E06D2F0E94B90286E06C2F0E94B90251
:1013E0008091A203F701E80FF11D60818F5F809368
:1013F000A20387E00E94B9022196C017D10740F3EB
:10140000DF91CF911F910F91FF90EF900895609120
:10141000030181E04DE051E025E00E94D4090895E8
:10142000DF93CF9300D000D0CDB7DEB7F8943091E2
:101430004A027894832F6AE00E94551A282F0E944E
:10144000551A482F822F0E94551A292F832F0E9448
:10145000551A992319F48AE08C8301C09C832223B6
:1014600019F48AE08A8301C02A83498385E48B8347
:1014700083E061E0AE014F5F5F4F24E00E94D4093A
:101480000F900F900F900F90CF91DF910895DF9301
:10149000CF9300D000D0CDB7DEB780E289839BE048
:1014A0009A8381E38B839C8381E061E0AE014F5F8F
:1014B0005F4F21E00E94D40980919901813079F435
:1014C00062E0AE014E5F5F4F21E00E94D40981E0EF
:1014D00063E0AE014D5F5F4F22E00E94D4090F90A0
:1014E0000F900F900F90CF91DF910895DF93CF93DE
:1014F00000D000D00F92CDB7DEB7DE011196E1E447
:10150000F1E085E001900D928150E1F760910401D6
:101510008CE0AE014F5F5F4F25E00E94D4090F9031
:101520000F900F900F900F90CF91DF91089580E072
:101530006CE40E94B90208958091180390911903F8
:10154000843B910554F080919A0390E0209116031A
:10155000309117038217930744F08091C9018823C3
:1015600071F481E08093C90108958091C901181632
:1015700024F480E06CE40E94B9021092C90108953D
:1015800080E062E40E94B90208958F929F92AF9228
:10159000BF92CF92DF92EF92FF920F931F93DF9350
:1015A000CF93CDB7DEB72F970FB6F894DEBF0FBE3F
:1015B000CDBFFE013B9685E0DF011D928A95E9F7DC
:1015C00080914602909147026EE170E00E94751A88
:1015D000CB01019797FF02C080E090E08E010F5F82
:1015E0001F4FB8014AE050E00E94241AF801019010
:1015F0000020E9F73197FE2EF01A80E0CF2CDD2491
:10160000C7FCD094F6E08F2E912C8C0E9D1E5801B5
:101610000BC0F501E00FF11F80810E94F305080D5A
:10162000191DF80180838E2D082F10E0E82EE39419
:101630000C151D0574F38093A20385E169E0AE01EA
:10164000455F5F4F25E00E94D40989E18F1969E069
:10165000A4012F2D0E94D4092F960FB6F894DEBF57
:101660000FBECDBFCF91DF911F910F91FF90EF90F3
:10167000DF90CF90BF90AF909F908F9008958F9202
:101680009F92AF92BF92CF92DF92EF92FF920F9311
:101690001F93DF93CF93CDB7DEB72E970FB6F89495
:1016A000DEBF0FBECDBF19821A821B821C828091C1
:1016B000AE019091AF018E010B5F1F4FB8014AE060
:1016C00050E00E94241AF80101900020E9F73197B8
:1016D000FE2EF01A80E0CF2CDD24C7FCD094AAE0C7
:1016E0008A2E912C8C0E9D1E58010BC0F501E00F27
:1016F000F11F80810E94F305080D191DF8018083F8
:101700008E2D082F10E0E82EE3940C151D0574F3C0
:101710008093A20385E166E0AE014F5F5F4F24E056
:101720000E94D40989E18F1966E0A4012F2D0E943F
:10173000D4098091AE019091AF011816190664F496
:1017400085E060E00E94B90286E062EC0E94B90286
:1017500087E06CE80E94B9028091AE019091AF01E0
:1017600097FF0CC085E060E00E94B90286E062EC61
:101770000E94B90287E06DE80E94B9028091AE0133
:101780009091AF01892B61F485E060E00E94B9027D
:1017900086E062EC0E94B90287E060E00E94B90234
:1017A0002E960FB6F894DEBF0FBECDBFCF91DF915E
:1017B0001F910F91FF90EF90DF90CF90BF90AF906F
:1017C0009F908F9008958F929F92AF92BF92CF92E9
:1017D000DF92EF92FF920F931F93DF93CF93CDB7DA
:1017E000DEB72B970FB6F894DEBF0FBECDBFDE017C
:1017F0001196EEE3F1E083E001900D928150E1F764
:101800008E010C5F1F4F8091140390911503B80156
:101810004AE050E00E94241AF80101900020E9F704
:101820003197FE2EF01A80E0CF2CDD24C7FCD09437
:10183000B8E08B2E912C8C0E9D1E58010BC0F5012B
:10184000E00FF11F80810E94F305080D191DF801BA
:1018500080838E2D082F10E0E82EE3940C151D05D3
:1018600074F38093A2038DE06EE0AE014F5F5F4F93
:1018700023E00E94D40980E18F196EE0A4012F2D8E
:101880000E94D4092B960FB6F894DEBF0FBECDBFD1
:10189000CF91DF911F910F91FF90EF90DF90CF904C
:1018A000BF90AF909F908F9008958F929F92AF922C
:1018B000BF92DF92EF92FF920F931F93DF93CF932C
:1018C000CDB7DEB728970FB6F894DEBF0FBECDBFF9
:1018D00019828AE08A838091A0019091A1018E01F2
:1018E0000D5F1F4FB8014AE050E00E94241AF80132
:1018F00001900020E9F73197E01B80E0EE2EFF24F5
:10190000E7FCF094480106E0A02EB12CAC0EBD1E01
:101910000BC0F401E00FF11F80810E94F3050A0D56
:101920001B1DF80180838D2D082F10E0D82ED39435
:101930000E151F0574F38093A2038091A00190916E
:10194000A1018E010A5F1F4F0A977CF46091030189
:1019500081E0AE014F5F5F4F21E00E94D4096091AA
:10196000030182E0A80121E005C06091030181E04C
:10197000A80122E00E94D4098091A2019091A301C4
:101980008E010D5F1F4FB8014AE050E00E94241AFB
:10199000F80101900020E9F73197E01B80E0EE2E7E
:1019A000FF24E7FCF094480116E0A12EB12CAC0E08
:1019B000BD1E0BC0F401E00FF11F80810E94F305F2
:1019C0000A0D1B1DF80180838D2D082F10E0D82EE5
:1019D000D3940E151F0574F38093A2038091A20186
:1019E0009091A3018E010A5F1F4F0A977CF46091CA
:1019F000030184E0AE014E5F5F4F21E00E94D409F5
:101A00006091030185E0A80121E005C06091030118
:101A100084E0A80122E00E94D40928960FB6F89429
:101A2000DEBF0FBECDBFCF91DF911F910F91FF9011
:101A3000EF90DF90BF90AF909F908F9008950F939D
:101A40001F93DF93CF93CDB7DEB72A970FB6F894E5
:101A5000DEBF0FBECDBF8E010F5F1F4FB8014AE042
:101A600050E00E94241AF80101900020E9F7319714
:101A7000E01B20E0FF27E7FDF095322F3F5F822F2C
:101A800090E08E179F0714F4232FF7CF2093A20323
:101A90002A960FB6F894DEBF0FBECDBFCF91DF916F
:101AA0001F910F910895AF92BF92CF92DF92EF9264
:101AB000FF920F931F93DF93CF93CDB7DEB76E974F
:101AC0000FB6F894DEBF0FBECDBFB82EA62ED42E13
:101AD000A42FB52FFD0101900020E9F73197CE2EFC
:101AE000C41A7E010894E11CF11C242F352FC90172
:101AF0008C0108C0F80181918F010E94F305F70164
:101B000081937F01802F8D198C15A0F38B2D6A2D69
:101B1000AE014F5F5F4F2C2D0E94D4096E960FB619
:101B2000F894DEBF0FBECDBFCF91DF911F910F9113
:101B3000FF90EF90DF90CF90BF90AF90089580918D
:101B40009801813071F4609106012091DF0130919C
:101B5000E001369527958EE0821B41EE51E00E9410
:101B6000530D0895EF92FF920F931F93DF93CF933E
:101B7000CDB7DEB764970FB6F894DEBF0FBECDBF0A
:101B8000F82EE62ECA018E010F5F1F4FB8014AE002
:101B900050E00E94241A8F2D6E2DA8010E94530D33
:101BA00064960FB6F894DEBF0FBECDBFCF91DF9124
:101BB0001F910F91FF90EF900895EF92FF920F9376
:101BC0001F93DF93CF93CDB7DEB72A970FB6F89464
:101BD000DEBF0FBECDBF20915303822F6AE00E946B
:101BE000551A382F822F0E94551A85E48F838091D1
:101BF0005403882309F48AE08887992319F48AE03A
:101C00008E8301C09E833D8319821A821B821C82AF
:101C10008E010B5F1F4F83E062E0A80124E00E9469
:101C2000D4098091570390915803B8014AE050E0DD
:101C30000E94241AF80101900020E9F77F0108941E
:101C4000E108F108E01AF10A83E063E0AE014F5FBA
:101C50005F4F24E00E94D40987E08E1963E0A80159
:101C60000E94530D2A960FB6F894DEBF0FBECDBF6B
:101C7000CF91DF911F910F91FF90EF900895BF9248
:101C8000CF92DF92EF92FF920F931F93DF93CF9348
:101C9000CDB7DEB764970FB6F894DEBF0FBECDBFE9
:101CA000C82EB62EFA017E010894E11CF11C04C076
:101CB000AE0DBF1D9C9331968E2F841B9491A82F3F
:101CC000B0E09923A9F7AE0DBF1D1C92F70101905A
:101CD0000020E9F73197DE2EDE18870107C0F801F2
:101CE00080810E94F305F80181938F01802F8E1966
:101CF0008D15A8F38C2D6B2DAE014F5F5F4F2D2DF1
:101D00000E94D40964960FB6F894DEBF0FBECDBF13
:101D1000CF91DF911F910F91FF90EF90DF90CF90C7
:101D2000BF9008951F93CF93DF93EC01A3E0B0E041
:101D300047C0FD01E459FD4F8081FD01E359FD4F8E
:101D40002081422F50E04D535040FD01E259FD4F9C
:101D50007081FD01E159FD4F10819A01F4E0359544
:101D60002795FA95E1F790E0CD97880F991F880F96
:101D7000991F282B392B2883613029F1E72FF0E0B8
:101D8000FD9734E0440F551F3A95E1F75070CF01AD
:101D90009595879595958795482B592B4983623062
:101DA00091F01496635086E0EE0FFF1F8A95E1F7DD
:101DB000F070812F90E0CD97E82BF92BEA832396E2
:101DC000662309F0B6CFDF91CF911F9108958091DE
:101DD0006E028635B1F480916D0281568093BA010E
:101DE0008091BA01843018F084E08093BA0184E4D1
:101DF00093E06AE043E02AE00E94920E81E0809343
:101E0000BB011092950108951F931091BA011230F1
:101E100009F486C0143009F4DBC0113009F09BC10D
:101E200080916E02813581F480E893E06BE143E0BC
:101E30002DE20E94920E8091800390E09093BD016C
:101E40008093BC011093C00180916E02843409F02C
:101E500082C182E093E061E443E021E40E94920EBB
:101E60008091180390911903843B910554F480915B
:101E70009A01813031F410929A01F8940E94BF10B7
:101E800078948091180390911903843B91057CF01C
:101E900080919A01882359F481E080939A01F89403
:101EA00080919701882311F40E94AF10789480915B
:101EB00004039091050366E170E00E94751A6E5F5D
:101EC0007F4F709345026093440280910603909186
:101ED000070366E170E00E94751A6A5F7F4F709396
:101EE00043026093420280910E0390910F039093FE
:101EF0004702809346028091160380934A028091A4
:101F0000290290912A02909349028093480280917D
:101F100014039091150390934D0280934C021BC1C2
:101F200080916E028F34A9F0813509F014C180E8E8
:101F300093E06CE143E02DE20E94920E80918003D9
:101F400090E09093BD018093BC0181E08093C0013B
:101F500002C185EF91E060E543E02DE20E94920E20
:101F600080913402992787FD9095029690934502BF
:101F70008093440280913502992787FD90950696BB
:101F8000909343028093420280912702909128020D
:101F9000909347028093460280912D0280934A02DB
:101FA0008091290290912A029093490280934802DD
:101FB000809132029091330290934D0280934C02B3
:101FC0008091260280934E0281E08093BF01C3C0BE
:101FD00080916E02843409F05AC082E093E061E49B
:101FE00043E021E40E94920E80911803909119031E
:101FF000843B910554F480919A01813031F4109220
:102000009A01F8940E94BF107894809118039091DF
:102010001903843B91057CF080919A01882359F43F
:1020200081E080939A01F89480919701882311F4BC
:102030000E94AF107894809104039091050366E1AB
:1020400070E00E94751A6E5F7F4F70934502609337
:102050004402809106039091070366E170E00E94BC
:10206000751A6A5F7F4F70934302609342028091BA
:102070000E0390910F039093470280934602809144
:1020800014039091150390934D0280934C0280911C
:102090006E028C3481F481E090E09093BD018093D6
:1020A000BC0181E08093C00182E893E069E143E0F4
:1020B0002DE20E94920E80916E028D3481F482E0B6
:1020C00090E09093BD018093BC0181E08093C001BA
:1020D00082E893E069E143E02DE20E94920E809154
:1020E0006E028E3481F483E090E09093BD01809382
:1020F000BC0181E08093C00182E893E069E143E0A4
:102100002DE20E94920E80916E028F3481F484E061
:1021100090E09093BD018093BC0181E08093C00169
:1021200082E893E069E143E02DE20E94920E809103
:102130006E02803581F485E090E09093BD0180933C
:10214000BC0181E08093C00182E893E069E143E053
:102150002DE20E94920E109295011F91089582E245
:1021600089B910BC80B91CBE909A28E92AB996E8B2
:1021700090BD82EC8BB921B99CBF82B9089582E2EF
:1021800089B910BC80B91CBE88E98AB926E820BD8F
:1021900092EC9BB980E981B92CBF92B90895DF9385
:1021A000CF93CDB7DEB72C970FB6F894DEBF0FBE36
:1021B000CDBF83E2898383E68A8385E78B838DE3C2
:1021C0008C838D838E838F83DE011196FD0120E049
:1021D00030E0AE01485F5F4F8191280F311DE41759
:1021E000F507D1F7C9019F7046E0959587954A9507
:1021F000E1F7835C88872F733070822F835C898737
:102200008DE08A879E01255F3F4F8C91159BFECF05
:1022100083B91196A217B307C1F72C960FB6F8949D
:10222000DEBF0FBECDBFCF91DF910895DF93CF9377
:10223000CDB7DEB72C970FB6F894DEBF0FBECDBF7B
:102240008BE189838A8385E58B838AEA8C831D826F
:10225000FE0131969E012A5F3F4F8081159BFECF84
:1022600083B93196E217F307C1F72C960FB6F894AD
:10227000DEBF0FBECDBFCF91DF910895DF93CF9327
:10228000CDB7DEB72A970FB6F894DEBF0FBECDBF2D
:1022900093E299838A836B83842F86958695835CEA
:1022A0008C8350E04370507064E0440F551F6A9572
:1022B000E1F7435C4D838DE38E838F83DE011196BE
:1022C000FD0120E030E0AE01485F5F4F8191280FB3
:1022D000311DE417F507D1F7C9019F7056E09595B8
:1022E00087955A95E1F7835C88872F733070822F2A
:1022F000835C89878DE08A879E01255F3F4F8C91A3
:10230000159BFECF83B91196A217B307C1F72A9682
:102310000FB6F894DEBF0FBECDBFCF91DF91089509
:102320005D9BFECF8DE68CB95D9BFECF8FE68CB9B1
:102330005D9BFECF89E68CB95D9BFECF8EE68CB9A6
:102340005D9BFECF8DE08CB95D9BFECF8EE38CB99B
:102350000895982F9F7082958F708A3010F4805D59
:1023600001C0895C5D9BFECF8CB99A3018F4892F2F
:10237000805D02C0892F895C5D9BFECF8CB908957A
:102380008A3010F4805D01C0895C5D9BFECF8CB902
:102390000895159BFECF83B908955D9BFECF8CB940
:1023A0000895662359F020E0FC01E20FF11DE08161
:1023B0005D9BFECFECB92F5F6217B0F708955D9B70
:1023C000FECF8EE38CB908951F920F920FB60F9235
:1023D00011242F933F938F939F93AF93BF93EF93CA
:1023E000FF932CB12093A30385B398E0892785BB85
:1023F0005D9BFECF2CB92D3059F080917F03E82FE3
:10240000F0E0E75AFC4F20838F5F80937F0359C031
:10241000E0917F03F0E0E75AFC4F20831092B70170
:102420001092B8011092B90130E020E090E03FC076
:102430002130B9F0213018F02230C1F524C0A32F8B
:10244000B0E0A75ABC4F8C91803211F421E023C038
:10245000E92FF0E08C91E958FC4F80839093B7010D
:1024600024C0A32FB0E0A75ABC4F8C91803211F446
:1024700022E011C0E92FF0E08C91E15AFD4F8083FA
:102480009093B80112C0A32FB0E0A75ABC4F8C9113
:10249000803219F423E090E009C0E92FF0E08C913C
:1024A000E05BFD4F80839093B9019F5F3F5F809118
:1024B0007F03831708F0BCCF81E08093B6011092B0
:1024C0007F03FF91EF91BF91AF919F918F913F91CA
:1024D0002F910F900FBE0F901F9018951F920F9283
:1024E0000FB60F9211248F939F93EF93FF9393B1A5
:1024F0009093A4039D3081F48091CA01813061F4EE
:10250000AB981092CA0180939501E0914F03F0E0DF
:10251000E459FD4F90832DC08091CA01882319F0A2
:10252000813039F514C0933241F4809195018823AC
:1025300021F481E08093CA01AB9A10924F038091FD
:102540004F03E82FF0E0E459FD4F90830CC0E09179
:102550004F03F0E0E459FD4F908380914F0385399C
:1025600030F480914F038F5F80934F0302C010922D
:10257000CA01FF91EF919F918F910F900FBE0F9025
:102580001F90189585B392E0892785BB0895909197
:102590009D01913019F485B3892785BB08951F9259
:1025A0000F920FB60F9211242F933F935F936F9367
:1025B0007F938F939F93AF93BF938091CC01909122
:1025C000CD01892B81F484B595B59093D301809387
:1025D000D2018EB58F7B8EBD81E090E09093CD01CE
:1025E0008093CC013AC084B595B59093D101809386
:1025F000D0012EB520642EBD2091D2013091D3019F
:102600001092CD011092CC01821B930B86569840FC
:102610006CE271E00E94611A7093CF016093CE0169
:102620006730710534F086E090E09093CF0180939D
:10263000CE012091CE013091CF01809102019927E6
:1026400087FD90952817390741F0263031052CF485
:102650002093020181E08093A401BF91AF919F91EB
:102660008F917F916F915F913F912F910F900FBE4E
:102670000F901F9018958091460290914702909379
:10268000A7018093A6018091A6019091A7012091B6
:10269000A8013091A901821B930B9093AB01809309
:1026A000AA018091A6019091A7019093A90180931E
:1026B000A8014091B2015091B3018091AA0190917B
:1026C000AB01E3E0880F991FEA95E1F79A0173E007
:1026D000220F331F7A95E1F7241B350B820F931FCE
:1026E00068E070E00E94751A7093B3016093B201C4
:1026F0002091B4013091B5014091B2015091B301E4
:10270000C90163E0880F991F6A95E1F7821B930B5B
:10271000840F951F68E070E00E94751A7093B501F0
:102720006093B4018091B4019091B5019093AF0191
:102730008093AE010E943F0B08958AE161E04EE470
:1027400051E022E00E94D4090895DF93CF9300D096
:102750000F92CDB7DEB7DE011196E0E5F1E083E040
:1027600001900D928150E1F7609104016F5F8EE05E
:10277000AE014F5F5F4F23E00E94D40960910401D6
:102780006F5F40912002509121028EE00E94B20DB5
:102790000F900F900F90CF91DF910895DF93CF931B
:1027A00000D00F92CDB7DEB7DE011196E3E5F1E080
:1027B00083E001900D928150E1F7609104018EE079
:1027C000AE014F5F5F4F23E00E94D4096091040186
:1027D00040912202509123028EE00E94B20D0F9090
:1027E0000F900F90CF91DF9108958F929F92BF929B
:1027F000CF92DF92EF92FF920F931F93DF93CF93CD
:10280000CDB7DEB72B970FB6F894DEBF0FBECDBFA6
:10281000DE011196E6E5F1E083E001900D92815032
:10282000E1F780914E028E010C5F1F4F90E0B801DE
:102830004AE050E00E94241AF80101900020E9F7D4
:102840003197BE2EB01AEE24FF24CB2CDD24C7FC1A
:10285000D09488E0882E912C8C0E9D1E0DC0F8011E
:10286000EE0DFF1D80810E94F305F401EE0DFF1DAA
:1028700080830894E11CF11CEC14FD0484F388E1CE
:1028800061E0AE014F5F5F4F23E00E94D4098BE10E
:102890008B1961E0A4012B2D0E94D4092B960FB651
:1028A000F894DEBF0FBECDBFCF91DF911F910F9186
:1028B000FF90EF90DF90CF90BF909F908F90089502
:1028C0008F929F92BF92CF92DF92EF92FF920F93DF
:1028D0001F93DF93CF93CDB7DEB76A970FB6F89407
:1028E000DEBF0FBECDBFFE01319686E0DF011D9237
:1028F0008A95E9F720912E0230912F0284E290E030
:10290000AC01249FC001259F900D349F900D112490
:1029100068EE73E00E94611ACB018E01095F1F4FC0
:10292000B8014AE050E00E94241AF801019000200A
:10293000E9F73197BE2EB01AEE24FF24CB2CDD240C
:10294000C7FCD09491E1892E912C8C0E9D1E0DC058
:10295000F801EE0DFF1D80810E94F305F401EE0DDC
:10296000FF1D80830894E11CF11CEC14FD0484F32A
:102970006091030185E1AE014F5F5F4F23E00E944C
:10298000D409609103018BE18B19A4012B2D0E94C6
:10299000D4096A960FB6F894DEBF0FBECDBFCF91B3
:1029A000DF911F910F91FF90EF90DF90CF90BF903C
:1029B0009F908F90089583E66FE644E60E943E1153
:1029C000F89428E088E190E00FB6F894A89581BDCE
:1029D0000FBE21BDFFCF1F939D998AC18091D40165
:1029E0008F5F8093D40111E01093D6018091D401C0
:1029F000853009F081C18091D801882309F08CC00D
:102A00001093D8011092D90184E064E00E94B902C9
:102A100083E061E041EE51E00E94530D83E063E00A
:102A200040E152E00E943F0E84E068E00E94B9025B
:102A300083E065E049E152E00E943F0E8091000191
:102A4000813029F484E165E045E452E004C084E18A
:102A500065E048E452E00E943F0E84E060E00E949E
:102A6000B90283E066E04DE152E00E943F0E8091A2
:102A70009701813029F484E166E045E452E004C026
:102A800084E166E048E452E00E943F0E83E067E0A4
:102A900043E252E00E943F0E80919801813029F478
:102AA00084E167E045E452E004C084E167E048E483
:102AB00052E00E943F0E83E068E04BE252E00E9449
:102AC0003F0E8091A501813029F484E168E045E45E
:102AD00052E004C084E168E048E452E00E943F0E06
:102AE00083E069E046E352E00E943F0E8091990145
:102AF000813029F484E169E045E452E004C084E1D6
:102B000069E048E452E00E943F0E83E06BE040E45D
:102B100052E00E943F0EEEC08091D901882349F512
:102B200084E068E00E94B90280910001882339F4B2
:102B30001093000184E165E045E452E006C0109284
:102B4000000184E165E048E452E00E943F0E2091DC
:102B50000001E199FECF81E090E09FBB8EBB2DBBD1
:102B60000FB6F894E29AE19A0FBE84E060E00E940A
:102B7000B9021091D901113049F584E068E00E9452
:102B8000B90280919701882339F41093970184E169
:102B900066E045E452E006C01092970184E166E0E9
:102BA00048E452E00E943F0E20919701E199FECF48
:102BB00080E090E09FBB8EBB2DBB0FB6F894E29AED
:102BC000E19A0FBE84E060E00E94B9028091D901D1
:102BD000823051F584E068E00E94B902809198014A
:102BE000882341F481E08093980184E167E045E423
:102BF00052E006C01092980184E167E048E452E098
:102C00000E943F0E20919801E199FECF82E090E072
:102C10009FBB8EBB2DBB0FB6F894E29AE19A0FBE14
:102C200084E060E00E94B9028091D901833051F5BF
:102C300084E068E00E94B9028091A501882341F4F4
:102C400081E08093A50184E168E045E452E006C09C
:102C50001092A50184E168E048E452E00E943F0E32
:102C60002091A501E199FECF87E190E09FBB8EBB4B
:102C70002DBB0FB6F894E29AE19A0FBE84E060E0B3
:102C80000E94B9028091D901843049F568E00E9420
:102C9000B90280919901882341F481E080939901E0
:102CA00084E169E045E452E006C01092990184E1B4
:102CB00069E048E452E00E943F0E20919901E199B9
:102CC000FECF8BE190E09FBB8EBB2DBB0FB6F8947F
:102CD000E29AE19A0FBE84E060E00E94B90280911E
:102CE000D901853049F41092D8010E94DB1404C048
:102CF0001092D4011092D6019C9913C19091D801E1
:102D0000913009F014C19093D7018091D5018F5F64
:102D10008093D5012091D501253009F008C110928A
:102D2000D5018091D901823009F469C0833030F433
:102D3000882371F0813009F0FAC035C0843009F47D
:102D4000AAC0843008F486C0853009F0F0C0C3C042
:102D50009093D90183E065E049E152E00E943F0E83
:102D600080910001813029F484E165E045E452E07E
:102D700004C084E165E048E452E00E943F0E84E034
:102D800068E00E94B90283E066E04DE152E00E94F3
:102D90003F0E80919701813019F484E166E0B3C061
:102DA00084E166E0B5C082E08093D90183E066E00B
:102DB0004DE152E00E943F0E80919701813029F44D
:102DC00084E166E045E452E004C084E166E048E462
:102DD00052E00E943F0E84E068E00E94B90283E066
:102DE00067E043E252E00E943F0E809198018130FB
:102DF00019F484E167E087C084E167E089C083E07B
:102E00008093D90167E043E252E00E943F0E809137
:102E10009801813029F484E167E045E452E004C080
:102E200084E167E048E452E00E943F0E84E068E0FD
:102E30000E94B90283E068E04BE252E00E943F0E3C
:102E40008091A501813019F484E168E05CC084E1DF
:102E500068E05EC084E08093D90183E068E04BE2E3
:102E600052E00E943F0E8091A501813029F484E157
:102E700068E045E452E004C084E168E048E452E0E0
:102E80000E943F0E84E068E00E94B90283E069E09E
:102E900046E352E03FC02093D90183E069E046E376
:102EA00052E00E943F0E80919901813029F484E123
:102EB00069E045E452E004C084E169E048E452E09E
:102EC0000E943F0E84E068E00E94B90283E06BE05C
:102ED00040E452E01FC01092D90183E06BE040E46F
:102EE00052E00E943F0E84E068E00E94B90283E055
:102EF00065E049E152E00E943F0E8091000181307F
:102F000029F484E165E045E452E004C084E165E031
:102F100048E452E00E943F0E84E060E00E94B90263
:102F200006C01092D5018091D6018091D7011F91E2
:102F30000895813061F4E199FECF80E090E09FBB7D
:102F40008EBB6DBB0FB6F894E29AE19A0FBE08955E
:102F5000DF93CF93CDB7DEB764970FB6F894DEBF9B
:102F60000FBECDBF20E0DE011196E199FECFE22F2A
:102F7000F0E0CF018D5F9F4F9FBB8EBBE09A8DB37A
:102F8000EA0FFB1F8083882311F02F5FEECFFD0136
:102F900001900020E9F79F01215030402A1B3B0B94
:102FA0003093E0012093DF0190E0AE014F5F5F4F6F
:102FB00009C0FD01EF51FE4FA40FB51F8C91808316
:102FC00011829F5FA92FB0E0A217B30790F3649618
:102FD0000FB6F894DEBF0FBECDBFCF91DF9108953D
:102FE000DF93CF93CDB7DEB760970FB6F894DEBF0F
:102FF0000FBECDBF80914C0290914D0290936B0219
:1030000080936A0280916A0290916B026FE070E097
:103010000E94611ADE011596AD016A1B9E01205FB8
:103020003F4FE62FEA0FF0E0E55BFD4FE491ED93B3
:10303000A217B307B1F76091070119821A821B82A8
:103040001C8289E02BE00E94D409609108018EE087
:10305000AE014F5F5F4F24E00E94D40960910801E8
:1030600040916A0250916B028FE00E94B20D60960F
:103070000FB6F894DEBF0FBECDBFCF91DF9108959C
:10308000DF93CF93CDB7DEB7E2970FB6F894DEBFEC
:103090000FBECDBFDE011796E9E5F1E087E00190B4
:1030A0000D928150E1F7DE011E96E0E6F1E089E045
:1030B00001900D928150E1F7DE015796E9E6F1E0CB
:1030C0008EE001900D928150E1F7DE011196E7E765
:1030D000F1E086E001900D928150E1F7DE019596D6
:1030E000EDE7F1E08EE001900D928150E1F7509113
:1030F0007703609178034091790380917A0320E00F
:1031000030E0803711F421E030E080E090E04C3690
:1031100011F481E090E02823392380E0583609F447
:1031200081E090E0653609F491E0892390E028235E
:103130003923232B79F0CE01079666E00E94D11146
:10314000CE010E9668E00E94D111CE0147966DE047
:103150000E94D111509177036091780340917903D7
:1031600080917A0320E030E0873711F421E030E0ED
:1031700080E090E04F3611F481E090E0282339237D
:1031800080E0533709F481E090E0683609F491E07B
:10319000892390E028233923232B19F180915F02A2
:1031A00090916002893481F4943471F4CE010196D7
:1031B00065E00E94D11181EE91E06091DF010E94F3
:1031C000D1118DE00E94CD1180915F02909160023B
:1031D000863739F4953629F4CE0185966CE00E9445
:1031E000D11180917703209178034091790390E089
:1031F000833709F491E080E0253609F481E09823D3
:10320000892F90E020E030E0443711F421E030E0F5
:1032100082239323892B09F442C080915F0290910D
:103220006002893409F03BC0943409F038C020E0D2
:103230001AC0FD01E05BFD4FE081E199FECF822FD6
:1032400090E08D5F9F4F9FBB8EBBEDBB0FB6F89498
:10325000E29AE19A0FBEFD01E05BFD4F8081AF5124
:10326000BE4F8C932F5F8091B901A22FB0E0281739
:1032700000F3E199FECFCD018D5F9F4F9FBB8EBBC9
:103280001DBA0FB6F894E29AE19A0FBEE22FF0E071
:10329000EF51FE4F1082B093E001A093DF015091F7
:1032A0007703609178034091790380917A0320E05D
:1032B00030E0853611F421E030E080E090E04337E3
:1032C00011F481E090E02823392380E0523709F49B
:1032D00081E090E0653609F491E0892390E02823AD
:1032E0003923232B11F00E94DB140E94DF11E29698
:1032F0000FB6F894DEBF0FBECDBFCF91DF9108951A
:103300001F920F920FB60F9211242F933F938F931A
:103310009F93EF93FF938091DB01882381F080914D
:10332000DB0190E00197E0918D01F0918E01E80FB3
:10333000F91F8FB1808381E08093DC0103C08FB1DE
:103340008093AA032091DB0180918B0130E09927C3
:1033500087FD9095821793075CF084E080938C0141
:1033600081E08093DC018091DB018093A90308C098
:10337000929A1092DA0181E08093DD011092DE01D1
:103380008091DB018F5F8093DB01FF91EF919F9133
:103390008F913F912F910F900FBE0F901F90189516
:1033A00082ED8DB90895813029F4613011F492983D
:1033B0000895929A0895982F8091DA018823C9F48C
:1033C000913009F492989093DA0181E08093DE01C4
:1033D000913069F486E080938B011092DB018AE0E2
:1033E00080938C019093DC018AEA8093A90380E0AA
:1033F00008958091DC01813071F480918C018150BD
:1034000080938C018F5F39F48091A9038FB910925A
:10341000DC0181E0089581E00895CF93DF93C0E05F
:10342000D0E0E0918D01F0918E01EC0FFD1F8081C5
:103430000E94A9112196C730D10599F78DE00E940D
:10344000CD11DF91CF910895FB019F01E8944230A7
:10345000C4F04532B4F44A3029F497FB1EF4909539
:1034600081959F4F642F77270E94611A805D8A3370
:103470000CF0895D8193CB010097A1F716F45DE212
:1034800051931082C9010C94451ADC01FC01672F8D
:1034900071917723E1F7329704C07C916D9370832B
:1034A0006291AE17BF07C8F30895991B79E004C075
:1034B000991F961708F0961B881F7A95C9F7809573
:1034C0000895AA1BBB1B51E107C0AA1FBB1FA6176B
:1034D000B70710F0A61BB70B881F991F5A95A9F7BD
:1034E00080959095BC01CD01089597FB092E072684
:1034F0000AD077FD04D0E5DF06D000201AF47095DD
:1035000061957F4F0895F6F7909581959F4F0895A7
:04351000F894FFCF5D
:103514000101030E0786010E0C5C00000A00004442
:103524000000230023005464665363655262005113
:1035340061005060005060005161005262005363AA
:10354400655464666768696A6B6B6A6968670000DA
:103554000053536353530203F50180030D0A0A1DFC
:1035640000000000000000000068656C70200D0081
:1035740073686F772049440D0073686F7720766510
:103584007273696F6E0D004944203D2000302E395E
:103594002E322E312E626574610D0009075203002C
:00000001FF
